:020000040000FA
:020000000528D1
:08000800AA2A00308B008316C8
:10001000831683120730990083169F018316FC30E4
:1000200085008312A101B501A801A701AA01A901B8
:10003000AC01BC01BF01C001AE01AD01B4012F286C
:10004000831D2F286400303084002030C100FF3031
:100050008000840FC10B28283030C100C20064002A
:1000600083160230810083120030A4002330A600E2
:100070005030A5000430A300592056225E224228A9
:10008000232242284B2181212118BD21A118C12101
:100090002119CE21211AA822A11AA92234190C2231
:1000A000422835078A0103398207512A5928A52891
:1000B00070280230AE00AD015E220F30BC00BC0FD4
:1000C0000530BD00A1172A30BE002608AA00250869
:1000D000A900A801A701C001AB0170280B210800ED
:1000E00000308A0040088207952800002A0E8228E6
:1000F0002A088228290E8228290882288B280000B5
:100100008B2800000F39BC00BC0F0530BD00A117C3
:100110002D30BE0095287121BC01BC0F0530BD00FB
:10012000A1131830BE00A111A11600308A00400CA6
:10013000C00FC00F8207423462342234623422344A
:100140004234003400346234623400308A00400C9F
:1001500082070000B228C128CA28D728E128EA2847
:1001600000000000AB172B081F396622AA00AB0A5B
:100170002B081F396622A9002B0A3F39AB00AB17A9
:1001800042341030A8072808D03E0318C82862342B
:10019000A8016234A80A2808063E8318D428280833
:1001A000DB3E0319D4282234F030A8052234103065
:1001B000A7072708A03E0318DE2862340F30A705E2
:1001C0006234A70A2708063E8318E7282234F03055
:1001D000A70522347121AB1FFE28AB032B081F3962
:1001E0009B0027086F22AB032B081F399B002808B0
:1001F0006F22AB0AAB0AA201512200342808A600E4
:10020000AA002708A500A9004530A4007121A20179
:100210005122122100342A30BE00080001308A0029
:100220003E088200A1171830BE000430BF0008004D
:10023000A1131830BE0008001F30BE00080068215E
:100240002330BE000800A1171230BE00A11D080017
:10025000702008002D30BE0008001830BE00BC0819
:10026000031D3829A11D0800A1171C30BE0008007D
:10027000BC0B3E29A1171C30BE000800A1172D3071
:10028000BE003C30BD0B49292A30BE000530BD0000
:100290007830742108003208B1000508B200320835
:1002A0003106B40432093105B30408003708B6003A
:1002B0000508B70037093605B804381F0800381399
:1002C000B71F3F2A4A2A381B4A22B81B3F22080080
:1002D0006030AF0001308506AF0B6C290130850618
:1002E0000800603074292030AF00B000013085066E
:1002F000AF0B76297B297C29B00B7A29350EA0001B
:1003000008000B1D08000B11211435222308FE3EA6
:1003100003192116A30B08000430A3008F29A11490
:10032000A40A2408A63E03189C29831898290800CB
:100330002408063EA4000800A4012115A50A2508EA
:10034000A63E0318AA298318A62908002508063EF8
:10035000A5000800A501A60A2608A63E0318BB2989
:100360008318B7292608DC3E0319A60108002608D1
:10037000063EA6000800A60108002110A11B0E21C0
:100380000800A110A11FA1160000AB302407031C18
:100390000800BF08031908007321080021112C0868
:1003A0003F396622AC0A2602031DE0292C083F399A
:1003B00066222502031DE0290230AE00AD015A225B
:1003C000AC0A2C083F396622AC0A2602031DEF292D
:1003D0002C083F3966222502031DEF296222AC0A50
:1003E0002C08E03E031DCF29AC01BF08031908000B
:1003F000BF0380307421080033126821013051207E
:10040000B500350EA0000800B3126821003051205D
:10041000B500350EA000080034113219162ABF01AC
:1004200068218830B9000030BA000800B9013A08E4
:10043000FE3E0319232A03182C2A3A085120B5003E
:10044000350EA0000800C001B5015920A115221CDD
:100450000510221805140800C001B501350EA000D2
:10046000221C05102218051408000310B90C031CE7
:100470000800BA0A10306821080033130800B813C6
:10048000FF30AE070318452AAD072E082D040319C7
:10049000622208003813AE0F0800AD0F0800622278
:1004A0000800221C562A582AA21400345A2200346A
:1004B000622200342214A214051408002214A2108F
:1004C000051408002210A2100510080083169B00D6
:1004D0001C141A088312080083169B000800831658
:1004E0009A008B139C131C1555309D00AA309D005B
:1004F0009C141C119C18792A9C1383120800080074
:100500008510822AC500C50DC5098510F0308316F7
:100510008500831285140430C6008E2A450805061E
:1005200002398506C50C450805060239C50C850645
:10053000C60B8E2A9B2A9C2A85109E2A9F2A56210A
:1005400008000F39063E8318073E2A3EC3007F2A63
:10055000080008000B19B02A8B18B22A0B18B42A0D
:0C0560000B1109008B1009000B100900A2
:084000000100060007000500A5
:02400E008031FF
:1042000000004500010000000500330005004700E4
:10421000110059001200050017005400180000009A
:1042200024000000240000002400000024000000FE
:1042300024000000240000002400000024000000EE
:00000001FF
